:100000000C9479040C94A1040C94A1040C94A10404
:100010000C94A1040C94A1040C94A1040C94A104CC
:100020000C94A1040C94A1040C94E80B0C94570CB0
:100030000C94A1040C94A1040C94A1040C94A104AC
:100040000C94A1040C94A1040C94A1040C94A1049C
:100050000C94A1040C94A1040C94A1040C94890E9A
:100060000C94A1040C94A1040C94A1040C94A1047C
:100070000C94A1040C94A1040C94A1040C94A1046C
:100080000C94D30E0C94A1040C94A1040C94A10420
:100090000C94A1040C94A1040C94A1040C94A1044C
:1000A0000C94A1040C94A1040C94A104084AD73B1D
:1000B0003BCE016E84BCBFFDC12F3D6C74319ABD37
:1000C00056833DDA3D00C77F11BED9E4BB4C3E915B
:1000D0006BAAAABE000000803F05A84CCDB2D44E4A
:1000E000B93836A9020C50B9918688083CA6AAAA4C
:1000F0002ABE000000803F0000000000003E5B4F71
:100100005B3E3E6B4F6B3E1C3E7C3E1C183C7E3C77
:10011000181C577D571C1C5E7F5E1C00183C180085
:10012000FFE7C3E7FF0018241800FFE7DBE7FF3015
:10013000483A060E2629792926407F050507407F83
:1001400005253F5A3CE73C5A7F3E1C1C08081C1CF6
:100150003E7F14227F22145F5F005F5F06097F01EC
:100160007F006689956A606060606094A2FFA294D7
:1001700008047E040810207E201008082A1C0808A5
:100180001C2A08081E101010100C1E0C1E0C3038F3
:100190003E3830060E3E0E06000000000000005FF4
:1001A00000000007000700147F147F14242A7F2A10
:1001B00012231308646236495620500008070300D2
:1001C000001C2241000041221C002A1C7F1C2A081E
:1001D000083E080800807030000808080808000081
:1001E00060600020100804023E5149453E00427FF5
:1001F000400072494949462141494D331814127F44
:100200001027454545393C4A4949314121110907E3
:100210003649494936464949291E00001400000064
:100220004034000000081422411414141414004136
:1002300022140802015909063E415D594E7C1211F3
:10024000127C7F494949363E414141227F4141412B
:100250003E7F494949417F090909013E41415173A6
:100260007F0808087F00417F41002040413F017F17
:10027000081422417F404040407F021C027F7F04DF
:1002800008107F3E4141413E7F090909063E415128
:10029000215E7F09192946264949493203017F0118
:1002A000033F4040403F1F2040201F3F4038403F19
:1002B000631408146303047804036159494D43002F
:1002C0007F4141410204081020004141417F040266
:1002D00001020440404040400003070800205454FD
:1002E00078407F28444438384444442838444428DB
:1002F0007F385454541800087E090218A4A49C782E
:100300007F0804047800447D40002040403D007F89
:100310001028440000417F40007C047804787C0869
:100320000404783844444438FC182424181824243D
:1003300018FC7C08040408485454542404043F4422
:10034000243C4040207C1C2040201C3C4030403C51
:1003500044281028444C9090907C4464544C4400B1
:100360000836410000007700000041360800020115
:100370000204023C2623263C1EA1A161123A404001
:10038000207A38545455592155557941215454787F
:1003900041215554784020545579400C1E52721218
:1003A00039555555593954545459395554545800A0
:1003B00000457C410002457D420001457C40F0291A
:1003C0002429F0F0282528F07C5455450020545469
:1003D0007C547C0A097F49324949493232484848AD
:1003E00032324A4848303A4141217A3A42402078F4
:1003F000009DA0A07D39444444393D4040403D3CEF
:1004000024FF2424487E4943662B2FFC2F2BFF0911
:1004100029F620C0887E0903205454794100004405
:100420007D413048484A32384040227A007A0A0AF0
:10043000727D0D19317D2629292F28262929292663
:1004400030484D4020380808080808080808382FA8
:1004500010C8ACBA2F102834FA00007B0000081432
:100460002A142222142A14089500220095AA005565
:1004700000AAAA55AA55AA000000FF00101010FFFC
:1004800000141414FF001010FF00FF1010F010F003
:10049000141414FC001414F700FF0000FF00FF14F4
:1004A00014F404FC141417101F10101F101F141440
:1004B000141F00101010F0000000001F101010108A
:1004C0001F10101010F010000000FF10101010107E
:1004D00010101010FF10000000FF140000FF00FFBC
:1004E00000001F10170000FC04F414141710171458
:1004F00014F404F40000FF00F7141414141414147A
:10050000F700F7141414171410101F101F141414EC
:10051000F4141010F010F000001F101F0000001F56
:1005200014000000FC140000F010F01010FF10FF89
:10053000141414FF141010101F00000000F010FF1E
:10054000FFFFFFFFF0F0F0F0F0FFFFFF0000000002
:1005500000FFFF0F0F0F0F0F38444438447C2A2A46
:100560003E147E02020606027E027E026355494167
:10057000633844443C04407E201E2006027E020272
:1005800099A5E7A5991C2A492A1C4C7201724C3086
:100590004A4D4D303048784830BC625A463D3E495D
:1005A0004949007E0101017E2A2A2A2A2A44445F01
:1005B000444440514A444040444A51400000FF01F5
:1005C00003E080FF000008086B6B08361236243603
:1005D000060F090F06000018180000001010003068
:1005E00040FF0101001F01011E00191D1712003CF0
:1005F0003C3C3C0000000000F0F89C8E8783878E16
:100600009CF8F00000FEFF0303030303070EFCF851
:100610000000FEFF0303030303070EFCF80000FFC6
:10062000FF00000000000000FFFF0000FEFF8383CA
:10063000838383C7EE7C380000F8FC0E07030303B6
:10064000070EFCF800003F7FE0C08080C0E07F3FE5
:10065000FFFF01010101010101FFFF0000FFFF0C8D
:100660000C0C0C1C3E77E3C100007FFFC0C0C0C073
:10067000C0E0703F1F00001F3F70E0C0C0C0E070CE
:100680003F1F00007FFFC1C1C1C1C1E3773E1C0015
:10069000001F3F70E0C0C0C0E0703F1F00000000BE
:1006A0000001FFFF01000000D5F08D14A1C881CF2B
:1006B000D9F1AF200046696E616C2053636F72659B
:1006C0003A0047414D45204F564552007800B80149
:1006D00032002A023200930232007003640000806C
:1006E0009600280064003C000080C80014006400EC
:1006F00028000080DC051400E8031400008090014D
:1007000032005802320020033200E8036400008007
:10071000546865204D616368696E65206172726915
:100720007665640A66726F6D2074686520766F69FD
:10073000642E0A0A497420646F6573206E6F7420FA
:10074000737065616B2E0A497420646F6573206E47
:100750006F7420736C6565702E0A0A4974206F6E81
:100760006C792068756E676572732E0A0A596F7509
:100770007220636F6E74726163740A6973207369A7
:100780006D706C653A0A4272696E672069742070F8
:100790006C616E6574732E0A0A446F6E2774206153
:1007A000736B20776865726520746865790A676F76
:1007B0002E2049742066656564732E0A0A2D2D2D3E
:1007C0002047414D45504C4159202D2D2D0A0A55A9
:1007D000736520442D50616420746F20666C792EFF
:1007E0000A5072657373204120746F2066697265C8
:1007F0002E0A5072657373204220746F20746F77D5
:100800002E0A0A4272696E6720706C616E6574739D
:1008100020746F0A546865204D616368696E6520B5
:10082000636F72652E005072657373204120746F80
:10083000205374617274004541544552004F524236
:10084000495400412067616D65206279204B6569DC
:100850007468204A616E65730050726573656E74CA
:10086000730053797A7967792D53797374656D7351
:1008700000B80B1E00D0071E00E8032800F4016436
:10088000000080080B0002020200000904000001C1
:1008900002020000052400100105240101010424C6
:1008A0000206052406000107058103100040090423
:1008B0000100020A000000070502024000000705CF
:1008C00083024000000403090412010002EF020148
:1008D00040412336800001010203014172647569C1
:1008E0006E6F204C4C430041726475626F7900005A
:1008F0004D0F11241FBECFEFDAE0DEBFCDBF11E0F8
:10090000A0E0B1E0E8E6F7E402C005900D92A4355E
:10091000B107D9F727E0A4E5B1E001C01D92A732E5
:10092000B207E1F714E0C9E7D4E004C02197FE0163
:100930000E94AC23C837D107C9F70E947A0F0C94E4
:10094000B2230C94000080916201089590E0E3ECE2
:10095000F2E091119FEF8FEF919391939193919387
:100960008150D0F70895E3ECF2E0A0E0B8E0008019
:100970000EBC8111012C1197A0FDFDCF0192B9F79A
:100980000DB40895480F592F511D1416150684F5FE
:10099000803891056CF597FF02C090E080E0413807
:1009A000510514F040E850E0481BFB01E770FF27B9
:1009B00021E001C0220FEA95EAF777FF02C0695FE4
:1009C0007F4FFB0133E0F595E7953A95E1F7F69512
:1009D000FE2FEE27F795E795E80FF91FED53FD4F32
:1009E000415030F08191DF011197822B8C93F8CF29
:1009F0000895FC018091C202882311F13FB7F89459
:100A000082E08093E9002091F200822F90E0181696
:100A1000190614F481E090E0882339F0289844E620
:100A20004093C1024091F1004083222339F020918C
:100A3000F200211103C02BE62093E8003FBF089588
:100A40008FEF9FEF08952FB7F89483E08093E9002C
:100A50009091E800892F807295FF04C09091F20078
:100A600080E4891B2FBF08958091B90281110DC0C8
:100A700082E08093B50284E08093B6021092B802BF
:100A80001092B70281E08093B90285EB92E008955D
:100A9000CF93DF931F92CDB7DEB76983DC01ED9171
:100AA000FC910280F381E02D41E050E0BE016F5FD8
:100AB0007F4F09950F90DF91CF91089583E0809348
:100AC000E9008091F200882319F08AE38093E8001E
:100AD00008950E94230590E00895CF93DF931F921D
:100AE000CDB7DEB7FC018485958597FD08C02FEF53
:100AF0003FEF358724870F90DF91CF910895CE0186
:100B000001960E94F904019719F4898190E0F3CFCE
:100B10008FEF9FEFF0CF0F931F93CF93DF931F9231
:100B2000CDB7DEB78C01FC018485958597FF0BC09E
:100B3000CE0101960E94F904019771F4898190E039
:100B4000F80195878487F801848595850F90DF915A
:100B5000CF911F910F9108958FEF9FEFF1CFFC017F
:100B60008485958597FD0BC09FB7F89482E08093AC
:100B7000E9008091F2009FBF90E0019608959FB731
:100B8000F89482E08093E9008091F2009FBF90E0AA
:100B900008954091AF025091B0022091AD02309182
:100BA000AE0242175307B4F49091E8009570E1F358
:100BB0009091E80092FD19C08093F1008091AF02FE
:100BC0009091B00201968F739927892B19F48EEFBB
:100BD0008093E8008091AF029091B00201969093CB
:100BE000B0028093AF0281E0089580E00895DF9223
:100BF000EF92FF920F931F93CF93DF93D82E8A012A
:100C0000EB017B01E40EF51ECE15DF0559F0D7FE92
:100C100012C0FE0184910E94C90521968111F4CF72
:100C20000FEF1FEFC801DF91CF911F910F91FF9040
:100C3000EF90DF9008958881EECF0F931F93CF93AD
:100C4000DF931F92CDB7DEB782E0898342E450E0A4
:100C500063E878E080E80E94F7050E943405DC0133
:100C600012960D911C910115110589F0D801ED9195
:100C7000FC910280F381E02DBE016F5F7F4FC801C0
:100C8000099597FD04C0F80100851185ECCF898195
:100C90000F90DF91CF911F910F910895615030F027
:100CA0002091F100FC0120830196F8CF289884E67A
:100CB0008093C1020895FC010E94F206319728F04A
:100CC00068517C4F8F4F9F4FF9CFAB01FC010E94C1
:100CD000F206641775078E079F07C8F308958F9271
:100CE0009F92AF92BF92CF92DF92EF92FF920F93BB
:100CF0001F93CF93DF936C017B018A0180912901BF
:100D0000882309F45AC08091C202882309F455C08F
:100D10008091B40280FF05C08091E00082608093E2
:100D2000E000E801B12C8AEFA82E93E0892E2AE397
:100D3000922E209711F4BB20C9F10E942305811146
:100D400008C0AA94AA20C9F181E090E00E945B0645
:100D5000F0CF8C171D0611F00CF08C2F9FB7F89474
:100D60008092E9002091E80025FD02C09FBFE1CFFD
:100D7000282F30E0C21BD30BF701815020F04191A6
:100D80004093F100FACFE20EF31EBB2021F09092C7
:100D9000E800B12CEBCF8091E80085FDE7CF909281
:100DA000E800BB24B394209709F3F3CF5D9884E661
:100DB0008093B302101611063CF081E090E0F6013A
:100DC0009383828310E000E0C801DF91CF911F91EF
:100DD0000F91FF90EF90DF90CF90BF90AF909F90DA
:100DE0008F900895A9EAB2E02FB7F8947D918D9184
:100DF0009C9166B52FBFA89B05C06F3F18F47F5F1D
:100E00008F4F9F4F22E0660F771F881F991F2A95EB
:100E1000D1F70895AF92BF92CF92DF92EF92FF92F7
:100E20000F931F93CF93DF936C017B018B01040F12
:100E3000151FEB015E01AE18BF08C017D10759F0AE
:100E40006991D601ED91FC910190F081E02DC601F0
:100E50000995892B79F7C501DF91CF911F910F91EA
:100E6000FF90EF90DF90CF90BF90AF9008952091CA
:100E70005B01E0915901F0915A01CF0102969093E4
:100E80005A0180935901222319F085919491089574
:100E9000808191810895CF92DF92EF92FF92CF935C
:100EA000DF930E943707811520E8920791F4809123
:100EB00071008D7F80937100109291004698479841
:100EC00010925801DF91CF91FF90EF90DF90CF907B
:100ED000089521E020935801813020E8920751F4D1
:100EE000809156019091570190935A018093590136
:100EF0000E94370797FD05C020915501222309F470
:100F000054C020915401211150C021E020935C0174
:100F1000EC01DF77209709F04BC081E080935D0101
:100F200046983FE9C32E3FE0D32EE12CF12CCAEFC7
:100F3000D0E0E0912107F09122070995811103C0CB
:100F400081E080935D0180915C01882329F080918C
:100F50005D01882309F43FC047980E943707009736
:100F6000F1F19C01DE010E94C81FDC01CB0129E0E8
:100F7000B595A795979587952A95D1F710929000EA
:100F80002AE020939100D0929900C092980080931B
:100F90005E0190935F01A0936001B0936101809125
:100FA00071008260809371008DCF10925C01B0CF90
:100FB0009E0150E040E060E472E48FE090E00E9427
:100FC000741F69017A0181E0C81AD108E108F108AB
:100FD00010925D01AECF4699BFCF479ABECF8FEF3B
:100FE0009FEFDC01CBCF9C01E1E7F0E090819D7F9A
:100FF000908381E080935B0130935A0120935901E3
:1010000030935701209356010C944B0790E00C94B9
:101010005B068FB18095807F669B88601C9B846097
:1010200008955C988EBD00000DB407FEFDCF5C9A5C
:1010300008953E9A3F9A81E08093620108959091CD
:101040009B02982329F490919C02982381E009F453
:1010500080E00895CF93C82F0E940908982F9C2301
:1010600081E09C1380E0CF91089580E00C94B3045C
:1010700080389105B8F460347105A0F490E121E066
:1010800061FD24E060FD220F62FD2295687F969F3E
:10109000D0011124A80FAD53BD4F0C90022A40FF80
:1010A00002260C9208952F923F924F925F926F9278
:1010B0007F928F929F92AF92BF92CF92DF92EF92E8
:1010C000FF920F931F93CF93DF93EC018B017A0173
:1010D0006901C61AD70AD7FE03C0D194C194D108BA
:1010E00047018C1A9D0A97FE03C091948194910840
:1010F0008C149D0454F49E2D8F2D7901292F382FA7
:101100009C2F8D2FE801092F182FEC16FD0654F4A3
:10111000902F812F8901292F382F9C2F8D2FE701A8
:10112000E92EF82E17012C1A3D0A2901401A510AFE
:1011300057FE03C0519441945108310137FE03C05A
:101140008FEF681A780A759467948FEF0217130768
:101150000CF481E0A82E880FBB08EC16FD06A4F065
:1011600041E0BE01C8018C149D0414F0B801CE0109
:101170000E9438086418750877FE04C00A0D1B1D0C
:10118000620C731C2196E9CFDF91CF911F910F91D3
:10119000FF90EF90DF90CF90BF90AF909F908F9097
:1011A0007F906F905F904F903F902F9008952F9277
:1011B0003F924F925F926F927F928F929F92AF92E7
:1011C000BF92CF92DF92EF92FF920F931F93CF9334
:1011D000DF9300D000D0CDB7DEB77C018B01242F88
:1011E00030E03C832B8381E090E05C01A21AB30ADB
:1011F0001901319421943108220C331CB901600F7C
:10120000711F41E0C7010E943808B8018B819C81A1
:10121000681B790B41E0C7010E94380841E0B80122
:101220008B819C818E0D9F1D0E94380841E0B80182
:10123000C7012B813C81821B930B0E943808D12C63
:10124000C12C81E090E09A8389832B813C81C21676
:10125000D3060CF05DC0B7FC09C0215031093C83B6
:101260002B8332E0230E311CA20CB31C8FEFC81A63
:10127000D80A29813A812E5F3F4F3A832983A20EF3
:10128000B31E37016C0C7D1C41E08B809C80800E6E
:10129000911EB401C3010E94380827014C185D0853
:1012A00041E0B401C2010E94380841E048018B814D
:1012B0009C81881A990AB401C3010E94380841E050
:1012C000B401C2010E9438084601800E911E41E01F
:1012D000B4016B807C806E0C7F1CC3010E943808B7
:1012E00041E0B40127012B813C81421A530AC2011B
:1012F0000E94380848018C189D0841E0B401C301E0
:101300000E94380841E0B401C2010E9438089DCF14
:101310000F900F900F900F90DF91CF911F910F9131
:10132000FF90EF90DF90CF90BF90AF909F908F9005
:101330007F906F905F904F903F902F9008952F92E5
:101340003F924F925F926F927F928F929F92AF9255
:10135000BF92CF92DF92EF92FF920F931F93CF93A2
:10136000DF9300D000D000D01F92CDB7DEB76D3034
:10137000D9F03090050140909F025090A002832D3B
:1013800090E09F838E836A3051F510929E021092F6
:101390009D0223E0880F991F2A95E1F7480E591EF8
:1013A0005092A00240929F0281E090E027960FB6F3
:1013B000F894DEBF0FBECDBFDF91CF911F910F918B
:1013C000FF90EF90DF90CF90BF90AF909F908F9065
:1013D0007F906F905F904F903F902F900895A090D6
:1013E0009D02B0909E0295E0699FB0011124FB011F
:1013F000E850FF4F3F016501212CF5E02F1629F140
:10140000C3010196F301F491F9833C01420128E004
:101410002A83898181708D8310E000E00315D0F468
:10142000F801EC0DFD1DFC83EB83F12CE12CE314A2
:1014300070F4B4016E0D7F1D4D818B819C810E94E3
:101440003808FFEFEF1AFF0AF2CF1982DFCF0F5FE4
:101450001F4FE4CF2981269529838A8181508A8371
:10146000EE81FF818E0E9F1E8111D3CF2394CE0E6D
:10147000DF1EF6E02F12C1CFC501329C800D911DF9
:10148000112490939E0280939D028ECF0F931F9301
:10149000CF93DF938C01D0E0C0E0F801EC0FFD1F8B
:1014A0006491662341F083E297E00E949F09892BB3
:1014B00011F02196F2CFCE01DF91CF911F910F91C4
:1014C0000895DF92EF92FF920F931F93CF93DF93D4
:1014D0007C01D22E8B01040F111DEB0177FF02C09E
:1014E000D0E0C0E0C8010134110514F080E490E0C0
:1014F000C817D9073CF44D2DBE01C7010E9438081A
:101500002196F0CFDF91CF911F910F91FF90EF9037
:10151000DF900895EF92FF920F931F93CF93DF9385
:101520007C018B01C42FD22F6034710510F40E940E
:10153000C204B8016D0F711D6150710960347105ED
:1015400020F44C2FC7010E94C20421E04D2FB801A6
:10155000C7010E94610AC7018C0F911D21E04D2F28
:10156000B8010197DF91CF911F910F91FF90EF90FC
:101570000C94610A2F923F924F925F926F927F92EA
:101580008F929F92AF92BF92CF92DF92EF92FF9293
:101590000F931F93CF93DF9300D000D0CDB7DEB76A
:1015A0006C015B01322E842F90E09C838B83440F6F
:1015B0004F5F681B790BC6010E94610A01E010E0D1
:1015C000EB81FC810E1B1F0B4F01919481949108BC
:1015D000880C991C66246394712CF12CE12C17FD66
:1015E0000AC08B819C8101979C838B8392E0890E3A
:1015F000911C080D191DEFEFEE1AFE0AF2E06F0EB6
:10160000711C060D171D2B80220C2394232D422DB7
:1016100025018B819C81481A590AB201C7018C0DA2
:101620009D1D0E94610AF501EE19FF09FA83E98305
:10163000232D462DBF018B819C818C0D9D1D0E9409
:10164000610A232D422DB201C6018E199F090E9405
:10165000610A232D462D69817A81C601EB81FC81C7
:101660008E1B9F0B0E94610A8B819C81E816F906F4
:101670000CF4B5CF0F900F900F900F90DF91CF919A
:101680001F910F91FF90EF90DF90CF90BF90AF90A0
:101690009F908F907F906F905F904F903F902F9092
:1016A0000895089590E080E008958F929F92AF9200
:1016B000BF920F931F93CF93DF93CDB7DEB7A19760
:1016C0000FB6F894DEBF0FBECDBF19A2423008F4AA
:1016D0004AE08E010F5D1F4F842E912CB12CA12C5E
:1016E000A50194010E94A61FE62FB901CA01EA30A4
:1016F00044F5E05DD801EE938D01232B242B252B9F
:1017000079F790E080E0109769F0FD0101900020EA
:10171000E9F73197AF014A1B5B0BBD0183E297E00C
:101720000E940A07A1960FB6F894DEBF0FBECDBF88
:10173000DF91CF911F910F91BF90AF909F908F90AD
:101740000895E95CD7CFCF92DF92EF92FF92CF93CB
:10175000DF936B017C016DE283E297E00E949F09B9
:10176000EC0166277727CB016C197D098E099F094B
:101770004AE00E94550B8C0F9D1FDF91CF91FF9087
:10178000EF90DF90CF900895BC01990F880B990BD3
:1017900097FD0C94A30B4AE00C94550BCF92DF926B
:1017A000EF92FF926B017C01C114D104E104F104BA
:1017B00041F00E94021FA70196010E94741F6B0155
:1017C0007C01C701B601FF90EF90DF90CF900895A4
:1017D0001F920F920FB60F9211248F939F938091B7
:1017E000E1009091E100937F9093E10083FF0FC0AF
:1017F0001092E90091E09093EB001092EC0092E3DC
:101800009093ED001092C20298E09093F00082FF56
:1018100022C093E09093E9009091F200992319F08F
:101820009AE39093E8009091B302992341F090914C
:10183000B30291509093B302911101C05D9A9091BF
:10184000C102992341F09091C10291509093C1023D
:10185000911101C0289A84FF18C08091E2008E7E09
:1018600081608093E2008091E1008F7E8093E100AF
:101870008091B4028E7E80618093B4029F918F919B
:101880000F900FBE0F901F90189580FFF7CF80919B
:10189000E2008E7E80618093E2008091E1008E7E86
:1018A0008093E1008091B4028E7E8160E5CF1F922B
:1018B0000F920FB60F921124CF92DF92EF92FF9208
:1018C0000F931F932F933F934F935F936F937F9348
:1018D0008F939F93AF93BF93EF93FF93CF93DF9338
:1018E000CDB7DEB76C97DEBFCDBF1092E900809117
:1018F000E80083FF25C068E0CE0145960E944E06B1
:1019000082EF8093E8008D8987FF39C09091E800CD
:1019100090FFFCCF982F907609F034C19E894F89B3
:10192000588D2F89F88C911131C0803861F58091E4
:10193000B2028093F1001092F1008EEF8093E800E4
:101940006C960FB6F894DEBF0FBECDBFDF91CF917E
:10195000FF91EF91BF91AF919F918F917F916F9187
:101960005F914F913F912F911F910F91FF90EF90B9
:10197000DF90CF900F900FBE0F901F9018959EEFA5
:101980009093E800C7CF1092F100D5CF913059F471
:101990008111D3CF4130510581F68091B2028D7F04
:1019A0008093B202CACF933049F48111C6CF41303F
:1019B000510519F68091B2028260F2CF953041F460
:1019C0008091E80080FFFCCF20682093E300B5CF32
:1019D000963009F0A9C00B8D1C8D22E01092E90011
:1019E0001092B0021092AF02F2122EC01092AE020C
:1019F0001092AD020E941D061F8299E09983FA821F
:101A000091E09E8390EA98879AEF99872091AF02A0
:101A10003091B002275F3F4F3C832B838D83109220
:101A2000E9001092B0021092AF021093AE02009340
:101A3000AD0249E050E0BE016F5F7F4F80E00E9441
:101A4000F7050E941D0679CF1093AE020093AD02F8
:101A50000E943405DC0112960D911C9101151105AF
:101A600009F451C1D801ED91FC910480F581E02D7C
:101A7000BE016B5E7F4FC8010995009709F03EC11A
:101A8000F80100851185EACFF3E0FF120EC08F89BF
:101A9000882309F440C0823061F440E867E087EEB3
:101AA00098E00E941A0F811148CF81E28093EB00E9
:101AB00047CF813029F440E86BE08BED98E0F1CF1F
:101AC000833099F70E943405DC011296ED90FC906A
:101AD0008E010F5F1F4F6801E114F10479F0D70107
:101AE000ED91FC910680F781E02DB801C7010995C1
:101AF000080F111DF701E084F184EECFD8011C928C
:101B0000F60101900020E9F73197BF016C197D09BA
:101B100040E0C601C6CF65EC78E0FB01449150E09F
:101B200080E80E94F70509CF973009F4BECF9830BE
:101B300021F481E08093F10000CF993009F0FDCECF
:101B4000837009F0B2CFEFE2F1E081E031E096E39B
:101B50002191222371F08093E9003093EB00DF01A3
:101B600011972C912093EC009093ED008F5F8730BC
:101B700079F78EE78093EA001092EA008F898093CC
:101B8000C202DBCE8B8D9C8D1092E9001092B002C8
:101B90001092AF029093AE028093AD02898D8111B5
:101BA00092C08E899D89913A49F4813209F07DCFA6
:101BB00047E050E062E271E080E0B3CF913209F09B
:101BC00074CF833269F48F89988DB0E0A0E0809360
:101BD0001E0190931F01A0932001B0932101ADCE6F
:101BE000803269F48091E80082FFFCCF67E082E2F6
:101BF00091E00E944E068BEF8093E8009ECE8232E9
:101C000009F09BCE8F8980932901EEEFFFE7859144
:101C100094918B3F9C4D51F1E0E0F8E080912201DE
:101C200090912301A0912401B0912501803B944023
:101C3000A105B105F1F48091290180FD1AC0EE3FA4
:101C40008AE0F80789F587E797E791838083809199
:101C500060008093B10288E19BE00FB6F894A895EC
:101C6000809360000FBE9093600067CEEEEFFAE0C5
:101C7000D5CF808191818737974709F05ECEA895AF
:101C8000809160008861809360008091B1028093B0
:101C90006000EE3F2AE0F20789F08091FE0A909101
:101CA000FF0A9183808349CE80819181873798078D
:101CB00051F29093FF0A8093FE0AC5CF1092FF0A5B
:101CC0001092FE0A3ACE0E943405DC0112960D9164
:101CD0001C910115110509F4E8CED801ED91FC9194
:101CE0000190F081E02DBE016B5E7F4FC801099528
:101CF000811123CEF80100851185EBCF1816190646
:101D00000CF41BCED2CEF1E0FF12BECE69EC78E02F
:101D100004CF0F920FB68F939F93EF93FF93809111
:101D2000A4028D5F8D3708F08D578093A402E5EAF9
:101D3000F2E080818E4F808391819F4F91838281D9
:101D40008F4F828383818F4F8383E9EAF2E0808122
:101D50008F5F808381818F4F818382818F4F8283C8
:101D600083818F4F83838FB18F6066991C9B8827F7
:101D70008F3681F48091A302981B963068F0E0E0E2
:101D8000F8E087E78083818388E180936000F093A7
:101D90006000FFCF9093A302FF91EF919F918F91ED
:101DA0000FBE0F9018951F920F920FB60F9211242D
:101DB0002F933F934F935F936F937F938F939F9353
:101DC000AF93BF93EF93FF9380915E0190915F017A
:101DD000A0916001B09161010097A105B10539F1B1
:101DE00020915D01211105C0369A20915C012111DD
:101DF000379A0197A109B109B7FD08C080935E0128
:101E000090935F01A0936001B0936101FF91EF9106
:101E1000BF91AF919F918F917F916F915F914F9102
:101E20003F912F910F900FBE0F901F9018950E9419
:101E30004B07ECCFEF92FF920F931F93CF93DF935B
:101E4000F82E192FE62E042F81E0860F880F0E94AE
:101E5000C90583E00E94C905CF2DD12FEC0EFD2EC0
:101E6000F11CCE15DF05B9F007FF13C0FE01849108
:101E70000E94C905182F80E00E94C9058123219680
:101E80008111EFCFDF91CF911F910F91FF90EF90D4
:101E900008958881EDCF81E0F5CFE3ECF6E0138281
:101EA000128288EE93E0A0E0B0E084839583A6835D
:101EB000B78389E391E0918380838FEF9FEF9587CC
:101EC0008487E3E2F7E0138212828BE491E091834E
:101ED000808383EA94E0909322078093210780E037
:101EE00090E89093200780931F0746983E9A479862
:101EF0003F9A0895CDB7DEB7A897DEBFCDBF7894DF
:101F000083E084BD83E085BD81E080936E00E1E8DD
:101F1000F0E083E08083E0E881E08083E1E983E032
:101F20008083E0E981E08083E1EC87E08083E3EC7B
:101F300081E08083E0EC82E08083E2EC81E08083DA
:101F4000EAE787E08083806880831092C202109263
:101F5000B2021092B4028091D70081608093D700C2
:101F600080EA8093D80089B5806189BD89B5826097
:101F700089BD09B400FEFDCF81E090E00E945B06C0
:101F80008091D8008F7C80618093D8008091E000A0
:101F9000807F8093E0008091E1008E7E8093E1005D
:101FA0008DE08093E200559A209A81EC80937C002A
:101FB00081EF85B987EE84B984E38BB984EF8AB960
:101FC000769A6E9880EF81BB10BA80E58CBD81E077
:101FD0008DBD85E00E9406085F9A85E00E94060894
:101FE0005C98E8EAF6E085918EBD00000DB407FE2E
:101FF000FDCFE53BC1F75C9A81E88093640081E006
:10200000809365000E94350880E80E942A08882392
:1020100081F085EA0E9411082E982F982D988091C2
:10202000640080628093640081E083BF889513BE62
:10203000FCCF84E00E942A088823B9F12D9884E817
:102040000E942A088823A1F02D9A88EC0E94060895
:102050002F986FEF82E090E00E94621F84EF91E082
:102060000E945B062F9A84E80E942A088111FBCF08
:1020700084E10E942A088823A1F02D9A88EC0E940E
:1020800006082E9860E082E090E00E94621F84EFD4
:1020900091E00E945B062E9A84E10E942A08811139
:1020A000FBCF88EC0E940608C4CF2D9A82E090E016
:1020B0000E945A1F882309F45AC00E94190881E01F
:1020C00090E00E945A1F182F147081FF0EC011114A
:1020D0002E98F1EF8F2E99249A9480E40E942A087A
:1020E000882309F449C02E9A2F9A82E30E94060899
:1020F0000E9409088111F9CF0E94190880E180939C
:1021000000010E94A6041092A00210929F02109259
:102110009E0210929D02E5E6F1E0FA8FE98F60E8F9
:1021200070E080E090E00E94CE0BA98DBA8D6C9398
:1021300060E470E080E090E00E94CE0BE98DFA8DC3
:1021400061833296FA8FE98F21EA31E02E173F073B
:1021500031F780916301882309F4B7C010926301BD
:1021600080E090E0892BA9F30E940000F2CF10924A
:1021700062013E983F98A3CF112331F004E080160E
:10218000910411F42E9A2F9881E00E94B304282D17
:102190002770722EC40163E0959587956A95E1F7E3
:1021A000BC017695762F66277795679550E040E0DD
:1021B0008E3F3FEF930791F1DB01AD53BD4F30E010
:1021C00020E0FA01E850FA4F7F01FB01ED5BFC4F84
:1021D0006F01F701E20FF31FE491F0E02F01072CEC
:1021E00002C0440C551C0A94E2F78F3F980739F05F
:1021F0005496BC905497B4285496BC925497772028
:1022000039F05601A20EB31EF50104890529048B8D
:102210002F5F3F4F119628353105D9F60196485A60
:102220005F4F60587F4F403B510509F0C1CF0E947E
:1022300035088FE00E940608FFEF8F1A9F0A09E118
:102240008016910409F049CF112311F02F9A2D988F
:1022500080E991E00E945B062D9A81E090E00E9467
:102260005A1F80FF42CF8AE090E00E945A1F9FEFE2
:10227000980F9E3F08F039CF22E330E030939E0262
:1022800020939D0228E330E03093A00220939F0228
:102290002AE030E03A832983682F83E297E00E94A6
:1022A0009F0949815A814F5F5F4F5A834983CA0111
:1022B0000E945A1FA981BA81509771F70E94350870
:1022C00088EE93E00E945B0610CF9091A50280916A
:1022D0006401392F381B832F20910001321748F4F5
:1022E0008F5F821708F03CCF81E083BF889513BED3
:1022F00037CF81E08093630190936401E9E2F2E0DB
:10230000808191810196808391830E94A60410921E
:10231000A00210929F0210929E0210929D02809144
:102320009C0280939B020E94090880939C028091EA
:10233000A1029091A2028230910509F434C148F4BF
:10234000009709F452C0019709F403C10E943508AF
:1023500007CF8430910509F45DC208F42DC20597BA
:10236000A9F788E00E941F08882351F082E090E0DE
:102370009093A2028093A10210929A021092990265
:1023800082E0809305018AE090E090939E02809322
:102390009D0280E190E09093A00280939F0282ECE6
:1023A00096E00E94460A81E08093050184E190E076
:1023B00090939E0280939D0288E290E09093A00209
:1023C00080939F0285EB96E00E94460A60919702F7
:1023D00070919802072E000C880B990B97FD02C094
:1023E0000C94B11E0E94A30BB1CF809199029091E1
:1023F0009A02019690939A02809399028C339105E8
:1024000009F06EC087EA0E94110881E798E00E94F7
:10241000F3078091990290919A02853B91052CF4E3
:1024200088E00E941F08882351F081E090E090939B
:10243000A2028093A10210929A02109299024091F6
:10244000990250919A025A8349834C3351050CF0FA
:102450004FC02AE430E0DA010E94A5232CE330E0EB
:1024600040E050E00E94741FDA01C9010A97A109F7
:10247000B10921E044E068E170E00E94BA0A2981D4
:102480003A81A6EBBFEF0E949D232CE330E040E0B1
:1024900050E00E94741FDA01C90186579F4FAF4F69
:1024A000BF4F21E046E068E170E00E94BA0A22E2F4
:1024B00030E0A981BA810E94A5232CE330E040E0FE
:1024C00050E00E94741FCA01B9016A507109810964
:1024D000910921E048E080E490E00E94BA0A36CFFA
:1024E0008134910509F095CF86EA0E94110891CFB9
:1024F00021E04CE068E170E080E490E00E94BA0ADC
:1025000020E04AE068E170E083E490E00E94BA0ACB
:1025100086E190E090939E0280939D0288E290E095
:102520009093A00280939F0282E698E00E94460A60
:10253000A8E2B0E0B0939E02A0939D0282E390E0F7
:102540009093A00280939F0289E598E00E94460A3A
:10255000FDCE8091990290919A02019690939A02F1
:1025600080939902893791052CF488E00E941F0816
:10257000882351F082E090E09093A2028093A10220
:1025800010929A021092990281E090E090939E023C
:1025900080939D028CE190E09093A00280939F0233
:1025A00083E498E0D3CF8091990290919A020196AA
:1025B00090939A028093990288E00E941F088823D2
:1025C00009F4A7C0109298021092970280ED97E04C
:1025D00090931B0180931A0183E090E0909319017E
:1025E0008093180184E690E0909317018093160180
:1025F00020E030E040E853E42093120130931301CF
:10260000409314015093150120930E0130930F0154
:102610004093100150931101109293021092940272
:10262000109295021092960210928F0210929002D0
:10263000109291021092920210928E026CE971E057
:1026400080E090E00E94CE0B6E5C7F4F8F4F9F4FDB
:102650000E946A2160930A0170930B0180930C0120
:1026600090930D016CE971E080E090E00E94CE0B48
:102670006E5C7F4F8F4F9F4F0E946A2160930601CF
:102680007093070180930801909309014EE552E091
:102690005A8349836CE971E080E090E00E94CE0BA0
:1026A0006E5C7F4F8F4F9F4F0E946A21A981BA8134
:1026B0006D937D938D939C9313976CE971E080E00B
:1026C00090E00E94CE0B6E5C7F4F8F4F9F4F0E9419
:1026D0006A21E981FA8164837583868397831086F2
:1026E00011861286138614861586168617867096AE
:1026F000FA83E983EE58F24069F610923B02109299
:102700004C0210925D0284E090E09093A2028093CC
:10271000A1028091990290919A028D32914064F0C9
:1027200083E090E09093A2028093A10280E490E085
:1027300090931D0180931C0182E08093050142E289
:1027400050E050939E0240939D0288E090E0909369
:10275000A00280939F028DE398E00E94460A82E2E5
:1027600090E090939E0280939D028AE190E0909386
:10277000A00280939F0287E398E00E94460A81E0CE
:10278000809305018091290290912A026CE370E008
:102790000E9475234E9708F0D9CD80E190E0909388
:1027A0009E0280939D0280E390E09093A00280932C
:1027B0009F0286E298E0CACE8091290280FD09C07E
:1027C00080911C0190911D01019790931D018093B0
:1027D0001C01A0911C01B0911D01BA83A983AC39E1
:1027E000BF4F2CF088E00E941F08882351F082E040
:1027F00090E09093A2028093A10210929A0210920C
:10280000990229813A813093A00220939F0280E1AE
:1028100097E09CCE80911A0190911B012091970224
:102820003091980228173907BCF020911801309197
:1028300019012830310534F42F5F3F4F30931901CF
:10284000209318018053984F90931B0180931A0195
:102850008EEF96E00E94F30788E00E941F0888230D
:1028600009F467C080913B02882311F40C94F41C96
:1028700080914C02882311F40C94F81C80915D0225
:10288000811157C082E090E021E1289FA001299F9B
:10289000500D1124455D5D4F5A83498381E0DA0173
:1028A00050968C938091120190911301A091140184
:1028B000B0911501FA0180839183A283B383809143
:1028C0000E0190910F01A0911001B091110184832C
:1028D0009583A683B783C0900101D0900201E09058
:1028E0000301F0900401C701B6010E94BB2020E063
:1028F00030E040EC50E40E948D22A981BA81189604
:102900006D937D938D939C931B97C701B6010E9495
:10291000FA2220E030E040EC50E40E948D22E98170
:10292000FA81648775878687978784EF96E00E948F
:10293000F30784E00E941F08882341F080918E02F3
:10294000882311F40C94FC1C10928E022BE232E0CE
:102950003E872D8719015FE0752ED10150968C912D
:102960005097882309F427C118962D913D914D91D8
:102970005C911B976D917D918D919C910E94D81FC8
:102980004B015C01F10180829182A282B382248595
:1029900035854685578564817581868197810E943A
:1029A000D81F6B017C01D1011496CD92DD92ED927E
:1029B000FC92179720E030E0A901C501B4010E9404
:1029C000B62087FD1DC020E030E040E054E4C501A2
:1029D000B4010E94802218169CF020E030E0A9018A
:1029E000C701B6010E94B62087FD0AC020E030E092
:1029F00040E054E4C701B6010E948022181614F486
:102A0000F101108A2EE532E03A832983D1015096F4
:102A10008C915097882309F4C2C0E981FA81208102
:102A20003181428153816D917D918D919C910E9464
:102A3000D71F4B015C01A981BA8114962D913D915C
:102A40004D915C911797F101648175818681978121
:102A50000E94D71F6B017C01A5019401C501B4013F
:102A60000E948D224B015C01A7019601C701B601AE
:102A70000E948D229B01AC01C501B4010E94D81FA8
:102A80000E94082320E030E040E051E40E94B6209C
:102A900087FF85C0D10150961C928AEE96E00E9475
:102AA000F30780919702909198024996909398022B
:102AB00080939702E981FA81C480D580E680F7800F
:102AC00080809180A280B38001EA11E0D8018D92CC
:102AD0009D92AD92BC921397F801C482D582E68292
:102AE000F78264E170E080E090E00E94CE0B6A50D3
:102AF0007109810991090E946A2120E030E040E2D9
:102B000051E40E94C020D80118966D937D938D9357
:102B10009C931B9764E170E080E090E00E94CE0BF4
:102B20006A507109810991090E946A2120E030E010
:102B300040E251E40E94C020F801648775878687CF
:102B40009787708A0F5E1F4F29E232E02017310706
:102B500009F0BCCF6CE971E080E090E00E94CE0B00
:102B60006E5C7F4F8F4F9F4F0E946A21A981BA816F
:102B70006D937D938D939C9313976CE971E080E046
:102B800090E00E94CE0B6E5C7F4F8F4F9F4F0E9454
:102B90006A21E981FA816483758386839783298119
:102BA0003A81205F3F4F3A8329834EE852E0421733
:102BB000530709F02BCF51E1250E311C8EE5281665
:102BC00082E0380609F0C9CEAEE5B2E0BC8FAB8F2B
:102BD0008D01D8012D913D914D915C912D8B3E8BB6
:102BE0004F8B588F609112017091130180911401E5
:102BF000909115010E94D71F6D837E838F839887E4
:102C0000D80114962D913D914D915C91179729878C
:102C10003A874B875C8760910E0170910F0180911C
:102C20001001909111010E94D71F69837A838B83D1
:102C30009C832D813E814F815885CA01B9010E9434
:102C40008D226B017C0129813A814B815C81CA0113
:102C5000B9010E948D229B01AC01C701B6010E94FF
:102C6000D81F0E9408236B017C0120E030E046E180
:102C700053E40E94B62087FF45C020E030E0A90160
:102C8000C701B6010E9480221816E4F5A70196013B
:102C90006D817E818F8198850E94C0202AE037ED6A
:102CA00043E25DE30E948D229B01AC01F801608547
:102CB0007185828593850E94D81FD80118966D93DF
:102CC0007D938D939C931B97A701960169817A81CF
:102CD0008B819C810E94C0202AE037ED43E25DE3B6
:102CE0000E948D229B01AC01F80164857585868563
:102CF00097850E94D81FD8011C966D937D938D9364
:102D00009C931F97F801408451846284738426E663
:102D100036E646E65FEBC301B2010E94B62087FDAE
:102D2000BCC626E636E646E65FE3C301B2010E9472
:102D30008022181634F446E6442E542C642C4FE3BB
:102D4000742ED8011C968D909D90AD90BC901F97CD
:102D500026E636E646E65FEBC501B4010E94B620E2
:102D600087FDA2C626E636E646E65FE3C501B40166
:102D70000E948022181634F426E6822E982CA82C65
:102D80002FE3B22E28E431EE4AE75FE3C301B2013C
:102D90000E948D222B013C01F801408651866286FB
:102DA000738628E431EE4AE75FE3C501B4010E946F
:102DB0008D224B015C01D8011C968D929D92AD92A3
:102DC000BC921F97A30192016D897E898F89988D8E
:102DD0000E94D81FF8016083718382839383A501C9
:102DE000940169857A858B859C850E94D81FD801BE
:102DF00014966D937D938D939C93179720E030E00C
:102E000040E051E4C701B6010E94B62087FF7DC0B3
:102E1000A70196016D817E818F8198850E94C020D7
:102E200020E030E040EC50E40E948D226093930259
:102E3000709394028093950290939602A701960155
:102E400069817A818B819C810E94C02020E030E0E2
:102E500040EC50E40E948D2260938F0270939002A8
:102E6000809391029093920210928E0280EE96E0EF
:102E70000E94F307F80180859185A285B385B0583B
:102E800080879187A287B38784859585A685B78536
:102E9000B05884879587A687B7878091160190914F
:102EA0001701499790931701809316011816190678
:102EB00064F1809118019091190101979093190183
:102EC0008093180124E630E0309317012093160117
:102ED00020E030E040E853E42093120130931301E6
:102EE000409314015093150120930E0130930F016C
:102EF00040931001509311011816190634F045E063
:102F000050E05093A2024093A102005F1F4F8EE851
:102F100092E08017910709F05CCEA1EAB1E0BE8B88
:102F2000AD8BBE83AD83AD81BE815096BC91B9831C
:102F3000BB2369F1ED81FE81208531854285538572
:102F400060817181828193810E94D81FAD81BE8191
:102F50006D937D938D939C9313971C962D913D912A
:102F60004D915C911F9714966D917D918D919C91DF
:102F700017970E94D81FED81FE8164837583868335
:102F80009783F981F150AD81BE815096FC932D81DC
:102F90003E812F5E3F4F3E832D8349E252E0421730
:102FA000530709F680918E02882309F4A3C080910B
:102FB0000A0190910B01A0910C01B0910D01898340
:102FC0009A83AB83BC832091060130910701409125
:102FD00008015091090129873A874B875C879C013A
:102FE000AD016091120170911301809114019091D3
:102FF00015010E94D71F4B015C0129853A854B853D
:103000005C8560910E0170910F018091100190918B
:1030100011010E94D71F2B013C01A5019401C5019C
:10302000B4010E948D226B017C01A3019201C301B6
:10303000B2010E948D229B01AC01C701B6010E9422
:10304000D81F0E9408236B017C0120E030E048EC8F
:1030500051E40E94802218160CF04CC020E030E0B1
:1030600048EC51E4C701B6010E94D71F698B7A8BE7
:103070008B8B9C8BA7019601C501B4010E94C020D7
:1030800029893A894B895C890E948D222DEC3CEC80
:103090004CEC5DE30E948D2229813A814B815C8159
:1030A0000E94D81F60930A0170930B0180930C015A
:1030B00090930D01A7019601C301B2010E94C020A7
:1030C00029893A894B895C890E948D222DEC3CEC40
:1030D0004CEC5DE30E948D2229853A854B855C8509
:1030E0000E94D81F60930601709307018093080126
:1030F0009093090120E030E040E853E460910A0138
:1031000070910B0180910C0190910D010E94D71FCD
:103110004B015C0120E030E040E853E4609106019F
:103120007091070180910801909109010E94D71FB9
:103130006B017C01A5019401C501B4010E948D229F
:103140004B015C01A7019601C701B6010E948D22C7
:103150009B01AC01C501B4010E94D81F0E94082345
:1031600020E030E040EC51E40E94B62087FF38C0F8
:1031700080919702909198028C599F4F909398025A
:103180008093970210928E028EEC96E00E94F307D5
:103190006CE971E080E090E00E94CE0B6E5C7F4FA6
:1031A0008F4F9F4F0E946A2160930A0170930B0119
:1031B00080930C0190930D016CE971E080E090E048
:1031C0000E94CE0B6E5C7F4F8F4F9F4F0E946A21F3
:1031D00060930601709307018093080190930901A1
:1031E00030918E023D8FBDEC8B2EBCEC9B2EBCE44F
:1031F000AB2EBEE3BB2EC12CD12C80E4E82EFE2CDE
:10320000332371F0FDEC8F2EFCEC9F2EFCE4AF2EEF
:10321000FDE3BF2EC12CD12CA0E8EA2EAFE3FA2E9D
:1032200080E80E942A088823A1F0A50194016091FA
:103230008F027091900280919102909192020E946F
:10324000D71F60938F0270939002809391029093A6
:10325000920280E10E942A088823A1F0A50194012E
:1032600060918F02709190028091910290919202F0
:103270000E94D81F60938F027093900280939102F6
:103280009093920280E20E942A088823A1F0A5016F
:1032900094016091930270919402809195029091B3
:1032A00096020E94D71F60939302709394028093BA
:1032B00095029093960280E40E942A088823A1F048
:1032C000A5019401609193027091940280919502FE
:1032D000909196020E94D81F60939302709394027B
:1032E000809395029093960246015701B7FAB094E5
:1032F000B7F8B09440909302509094026090950279
:10330000709096029201A301C501B4010E9480222F
:1033100018160CF4D0C39201A301C701B6010E9494
:10332000B62087FF02C02601370140918F024987EE
:1033300050919002598B809191028AA390919202B0
:103340009E8F9A01AC01C501B4010E94802218161B
:103350000CF4B4C3298539894AA15E8DC701B60131
:103360000E94B62087FF04C0C986D98AEAA2FE8ED1
:1033700023E333E343E75FE3B201C3010E948D22FD
:1033800069837A838B839C83609393027093940206
:10339000809395029093960223E333E343E75FE340
:1033A000698579898AA19E8D0E948D222B013C011D
:1033B00040928F025092900260929102709292021B
:1033C0002091120130911301409114015091150187
:1033D00069817A818B819C810E94D81F4B015C019D
:1033E00020E030E040E051E40E94B62087FD6BC34E
:1033F00020E030E04CEF53E4C501B4010E9480228C
:10340000181634F4812C912CECEFAE2EE3E4BE2E92
:103410008092120190921301A0921401B0921501B2
:1034200020910E0130910F01409110015091110136
:10343000C301B2010E94D81F6B017C0120E030E083
:1034400040E051E40E94B62087FD43C320E030E015
:103450004CEF53E4C701B6010E948022181634F4E1
:10346000C12CD12C6CEFE62E63E4F62EC0920E0137
:10347000D0920F01E0921001F092110120E030E0B3
:10348000A90169817A818B819C810E948022181612
:103490000CF025C32DEC3CEC4CEC5DE369817A81AA
:1034A0008B819C810E94802218160CF424C320E09A
:1034B00030E0A901C301B2010E94802218160CF06D
:1034C0002BC32DEC3CEC4CEC5DE3C301B2010E943C
:1034D000802218160CF40FC320E030E040E852E4DC
:1034E000C501B4010E94D71F0E9432214B0120E088
:1034F00030E040E052E4C701B6010E94D71F0E94AD
:1035000032212B01CB01940197FE02C02F5F3F4F68
:1035100035952795EE24FF24E21AF30A620197FFFE
:1035200003C0AFEFCA1ADA0AD594C794D194C194F4
:10353000D108E5E6F1E0FA83E983A981BA818C91AB
:103540008E0D9F2D911D60E870E00E948923FC0183
:103550009C01A981BA8111968C918C0D9D2D911D94
:1035600060E470E00E94892397FF02C0805C9F4F57
:10357000F7FF03C09F0120583F4F41E0BC01C90144
:103580000E943808E981FA813296FA83E983298D0D
:103590003A8DE217F30789F680E091E06C01C418D8
:1035A000D5087C01E818F90840E1B601C7010E947E
:1035B000D7086091290270912A0290E080E00E9471
:1035C00068212DEC3CEC4CEC5DE30E948D220E94C6
:1035D000FA2220E030E040E850E40E948D2220E012
:1035E00030E040E051E40E94D81F0E943921462F6C
:1035F000B601C7010E94D708B201550C880B990B80
:103600000E946A212B013C01AC019B0160910601E3
:103610007091070180910801909109010E94D71FC4
:103620000E94322169877A878B879C87B401990C25
:10363000880B990B0E946A2169837A838B839C8310
:103640009B01AC0160910A0170910B0180910C010A
:1036500090910D010E94D71F0E943221698B7A8BB5
:103660008B8B9C8B21E048E069857A8589899A89D2
:103670000E94BA0A4EE552E05FA34EA329813A8127
:103680004B815C81AEA1BFA16D917D918D919C918B
:103690000E94D71F0E9432216B01A3019201EEA16B
:1036A000FFA164817581868197810E94D71F0E9446
:1036B00032214B0164507109C601049728E048E0AB
:1036C0000E948A0A41E0B401C6010E9438082EA176
:1036D0003FA1205F3F4F3FA32EA30217130771F6B0
:1036E000AD85BE8550968C915097882309F45DC0B6
:1036F000A301920114966D917D918D919C911797E4
:103700000E94D71F4B015C0129813A814B815C816A
:10371000ED85FE8560817181828193810E94D71F32
:103720006B017C0120E030E040E05FE3AD85BE85C9
:103730001C966D917D918D919C911F970E948D2279
:103740009B01AC01C501B4010E94D71F0E94322128
:103750006E8F7F8F88A399A320E030E040E05FE385
:10376000ED85FE8560857185828593850E948D2219
:103770009B01AC01C701B6010E94D71F0E943221F4
:103780006AA37BA38CA39DA3C501B4010E9432212F
:103790004B01C701B6010E943221CB012E8D3F8D16
:1037A0004AA15BA1B4010E9453082D853E852F5E7E
:1037B0003F4F3E872D872216330609F091CFAD8902
:1037C000BE8950968C915097882301F1A3019201F4
:1037D00014966D917D918D919C9117970E94D71FA2
:1037E0000E9432216B0129813A814B815C81ED89F4
:1037F000FE8960817181828193810E94D71F0E941E
:103800003221CB0141E0B6010E9438082D893E8962
:103810002F5E3F4F3E8B2D8B4D815E8142175307AC
:1038200071F60D8D002371F08091290280FD0AC090
:1038300029853A8549895A8960E270E080E490E000
:103840000E945308C0900101D0900201E090030152
:10385000F090040120E030E040E250E4C701B601FE
:103860000E94D71F4B015C010E94FA2220E030E049
:1038700040EC50E40E948D2220E030E040E052E431
:103880000E94D81F0E9432216D837E838F83988788
:10389000C501B4010E94BB2020E030E040EC50E4C0
:1038A0000E948D2220E030E040E852E40E94D81FC0
:1038B0000E9432216D877E878F87988B20E030E0D1
:1038C00040E250E4C701B6010E94D81F4B015C01E1
:1038D0000E94FA2220E030E040EC50E40E948D2269
:1038E00020E030E040E052E40E94D81F0E943221E4
:1038F0002B01C501B4010E94BB2020E030E040EC68
:1039000050E40E948D2220E030E040E852E40E9422
:10391000D81F0E94322169837A838B839C83C701DD
:10392000B6010E94FA2220E030E040EC50E40E9410
:103930008D2220E030E040E052E40E94D81F0E9437
:1039400032214B01C701B6010E94BB2020E030E0CC
:1039500040EC50E40E948D2220E030E040E852E448
:103960000E94D81F0E9432216B01920149815A8125
:10397000B401C6010E9453082D813E814D855E85AC
:10398000B20189819A810E9453089401A6016D8138
:103990007E818D859E850E94530826E044E36AE37C
:1039A00070E090E080E00E948A0A00911601109178
:1039B000170117FF02C00F5F1F4F15950795EE24E3
:1039C000E394F12C11270F5F1F4FE016F1060CF066
:1039D000AEC021E044E06BE370E0C7010E94610AE1
:1039E0002FEFE21AF20AF1CF90E080E00C94441439
:1039F00081E090E00C944414209112013091130165
:103A0000409114015091150160910A0170910B01D0
:103A100080910C0190910D010E94D71F4B015C0118
:103A200020910E0130910F01409110015091110130
:103A30006091060170910701809108019091090140
:103A40000E94D71F6B017C01A5019401C501B4013F
:103A50000E948D224B015C01A7019601C701B601AE
:103A60000E948D229B01AC01C501B4010E94D81FA8
:103A70000E94082320E030E040E252E40E94B62099
:103A800087FD02C00C94A61481E080938E0281E72A
:103A900098E00E94F3070C94A61436E6432E542CAB
:103AA000642C3FEB732E4DC996E6892E982CA82CDA
:103AB0009FEBB92E67C92401350137CC8986998AD5
:103AC000AAA2BE8E55CC812C912CA12C71E4B72ECC
:103AD0009FCCC12CD12CE12C51E4F52EC7CC2DEC80
:103AE0003CEC4CEC5DEB69817A818B819C810E947E
:103AF000B62087FFDCCC29813A814B815C81C301F0
:103B0000B2010E94572060930101709302018093DB
:103B1000030190930401E0CC2DEC3CEC4CEC5DEB0C
:103B2000C301B2010E94B62087FFD6CCE4CF88E360
:103B300090E090939E0280939D029093A0028093C8
:103B40009F028CEC96E00E94460A809118019091A9
:103B500019010E94C40B10929E0210929D021092B5
:103B6000A00210929F0280919702909198020E9469
:103B7000C40B00E610E020E040E270E060E0C80125
:103B80000E94610A0F5F1F4F00381105A1F720E264
:103B900040E270E060E080E690E00E948A0A20E166
:103BA00030E041E750E060E170E08FE690E00E9495
:103BB000530821E130E040E750E06FE070E080E73B
:103BC00090E00E9453088091290290912A0264E1BA
:103BD00070E00E9475230A97D0F520E030E040E8BD
:103BE0005DE3609106017091070180910801909159
:103BF00009010E948D2220E030E0A9010E94D81F17
:103C00000E9432214B0120E030E040E85DE360910A
:103C10000A0170910B0180910C0190910D010E949D
:103C20008D2220E030E040EC52E40E94D81F0E9438
:103C300032216B0121E042E0B401C6010E94610A19
:103C4000C601019621E042E0B4010E94610A20E031
:103C500030E040E85DE360910E0170910F018091CA
:103C60001001909111010E948D2220E030E0A90105
:103C70000E94D81F0E9432216B0120E030E040E812
:103C80005DE3609112017091130180911401909194
:103C900015010E948D2220E030E040EC52E40E94A9
:103CA000D81F0E943221CB0141E0B6010E943808A2
:103CB0008091290290912A026EE170E00E947523A2
:103CC0000F9710F00C94A61120E030E040E85DE37F
:103CD000AB8DBC8D6D917D918D919C910E948D22BB
:103CE00020E030E040EC52E40E94D81F0E943221D4
:103CF0006B01CB01815691094D9728F520E030E00A
:103D000040E85DE3EB8DFC8D648175818681978150
:103D10000E948D2220E030E0A9010E94D81F0E945D
:103D200032214B01CB0101974D9768F421E042E02D
:103D3000B401C6010E94610AC601019621E042E079
:103D4000B4010E94610A2B8D3C8D205F3F4F3C8F58
:103D50002B8F4EA15FA14217530709F0B5CF0C94EA
:103D6000A6114AE00E94550B0C94A6118F929F92C7
:103D7000AF92BF92CF92DF92EF92FF92CF93DF93F9
:103D8000EC01688179818A819B81611571058105CA
:103D9000910521F464E279ED8BE597E02DE133EFB5
:103DA00041E050E00E94741F49015A019B01AC019F
:103DB000A7EAB1E40E94931F6B017C01ACEEB4EF63
:103DC000A50194010E94A11FC60ED71EE81EF91E70
:103DD000F7FE06C081E0C81AD108E10880E8F80AB9
:103DE000C882D982EA82FB82C701B6019F77DF9140
:103DF000CF91FF90EF90DF90CF90BF90AF909F90CA
:103E00008F9008958F929F92AF92BF92CF92DF9240
:103E1000EF92FF9260912A0170912B0180912C0109
:103E200090912D01611571058105910521F464E2E0
:103E300079ED8BE597E02DE133EF41E050E00E9412
:103E4000741F49015A019B01AC01A7EAB1E40E9429
:103E5000931F6B017C01ACEEB4EFA50194010E94AD
:103E6000A11FC60ED71EE81EF91EF7FE06C081E090
:103E7000C81AD108E10880E8F80AC0922A01D09255
:103E80002B01E0922C01F0922D01C701B6019F7722
:103E9000FF90EF90DF90CF90BF90AF909F908F906A
:103EA000089560932A0170932B0180932C019093C5
:103EB0002D010895F999FECF92BD81BDF89A9927F9
:103EC00080B50895262FF999FECF92BD81BDF89A4D
:103ED000019700B4021639F01FBA20BD0FB6F8944E
:103EE000FA9AF99A0FBE0895052E97FB1EF40094D6
:103EF0000E948B1F57FD07D00E94A61F07FC03D00E
:103F00004EF40C948B1F50954095309521953F4F62
:103F10004F4F5F4F089590958095709561957F4FB5
:103F20008F4F9F4F08950E94C81FA59F900DB49F6B
:103F3000900DA49F800D911D11240895B7FF0C943E
:103F4000931F0E94931F821B930B0895A1E21A2EC8
:103F5000AA1BBB1BFD010DC0AA1FBB1FEE1FFF1F2D
:103F6000A217B307E407F50720F0A21BB30BE40B7D
:103F7000F50B661F771F881F991F1A9469F76095C4
:103F80007095809590959B01AC01BD01CF0108957E
:103F9000A29FB001B39FC001A39F700D811D11248A
:103FA000911DB29F700D811D1124911D08955058CF
:103FB000BB27AA270E94EF1F0C9432220E94F921EE
:103FC00038F00E94002220F039F49F3F19F426F4C3
:103FD0000C94CF210EF4E095E7FB0C94C921E92F56
:103FE0000E94572258F3BA17620773078407950790
:103FF00020F079F4A6F50C9479220EF4E0950B2EBE
:10400000BA2FA02D0B01B90190010C01CA01A0012A
:104010001124FF27591B99F0593F50F4503E68F185
:104020001A16F040A22F232F342F4427585FF3CFC6
:10403000469537952795A795F0405395C9F77EF497
:104040001F16BA0B620B730B840BBAF09150A1F0E0
:10405000FF0FBB1F661F771F881FC2F70EC0BA0F66
:10406000621F731F841F48F4879577956795B795EE
:10407000F7959E3F08F0B0CF9395880F08F09927E9
:10408000EE0F9795879508950E94F92160F080E8DA
:1040900091E009F49EEF0E94002228F040E851E0F0
:1040A00071F45EEF0CC00C94CF210C947922E92FAF
:1040B000E0780E94572240F3092E052AB1F3261713
:1040C00037074807590738F00E2E07F8E02569F042
:1040D000E025E0640AC0EF6307F8009407FADB010B
:1040E000B9019D01DC01CA01AD01EF930E94D72007
:1040F0000E9432220E9487205F91552339F02BEDD8
:104100003FE049E450FD49EC0C94D81F0895DF933B
:10411000DD27B92FBF7740E85FE31616170648077B
:104120005B0718F4D92F0E9485229F938F937F936A
:104130006F930E944823ECEAF0E00E94D2210E9493
:1041400032222F913F914F915F910E94A022DD2357
:1041500051F09058A2EA2AED3FE049EC5FE3D078B5
:104160005D270E94EF1FDF910C9432220E94A5214F
:1041700008F481E008950E940922E3950C944322FB
:104180000E94D4200C9432220E94002258F00E94F7
:10419000F92140F029F45F3F29F00C94C921511115
:1041A0000C947A220C94CF210E94572268F3992311
:1041B000B1F3552391F3951B550BBB27AA27621723
:1041C0007307840738F09F5F5F4F220F331F441F30
:1041D000AA1FA9F335D00E2E3AF0E0E832D0915064
:1041E0005040E695001CCAF72BD0FE2F29D0660F51
:1041F000771F881FBB1F261737074807AB07B0E894
:1042000009F0BB0B802DBF01FF2793585F4F3AF099
:104210009E3F510578F00C94C9210C947A225F3F9F
:10422000E4F3983ED4F3869577956795B795F7951F
:104230009F5FC9F7880F911D9695879597F9089507
:10424000E1E0660F771F881FBB1F621773078407A3
:10425000BA0720F0621B730B840BBA0BEE1F88F7B2
:10426000E09508950E9439216894B1110C947A2246
:1042700008950E945F2288F09F5798F0B92F9927E0
:10428000B751B0F0E1F0660F771F881F991F1AF041
:10429000BA95C9F714C0B13091F00E947922B1E00B
:1042A00008950C947922672F782F8827B85F39F00A
:1042B000B93FCCF3869577956795B395D9F73EF4DA
:1042C00090958095709561957F4F8F4F9F4F089582
:1042D000E89409C097FB3EF49095809570956195A0
:1042E0007F4F8F4F9F4F9923A9F0F92F96E9BB2756
:1042F0009395F695879577956795B795F111F8CFD2
:10430000FAF4BB0F11F460FF1BC06F5F7F4F8F4F3C
:104310009F4F16C0882311F096E911C0772321F032
:104320009EE8872F762F05C0662371F096E8862FCA
:1043300070E060E02AF09A95660F771F881FDAF721
:10434000880F9695879597F90895990F0008550F4E
:10435000AA0BE0E8FEEF16161706E807F907C0F00B
:1043600012161306E407F50798F0621B730B840B13
:10437000950B39F40A2661F0232B242B252B21F4ED
:1043800008950A2609F4A140A6958FEF811D811D8D
:10439000089597F99F6780E870E060E008959FEFC7
:1043A00080EC0895DF93CF931F930F93FF92EF92CA
:1043B000DF927B018C01689406C0DA2EEF010E9427
:1043C000A022FE01E894A591259135914591559142
:1043D000A6F3EF010E94EF1FFE019701A801DA94F6
:1043E00069F7DF90EF90FF900F911F91CF91DF91D0
:1043F000089500240A94161617061806090608954B
:1044000000240A94121613061406050608950C9447
:10441000CF210E945F22D8F3E894E0E0BB279F57AA
:10442000F0F02AED3FE049EC06C0EE0FBB0F661F2F
:10443000771F881F28F0B23A62077307840728F0B5
:10444000B25A620B730B840BE3959A9572F780381E
:1044500030F49A95BB0F661F771F881FD2F79048DC
:104460000C944E23092E0394000C11F4882352F06F
:10447000BB0F40F4BF2B11F460FF04C06F5F7F4F90
:104480008F4F9F4F0895EF93E0FF07C0A2EA2AEDF8
:104490003FE049EC5FEB0E94EF1F0E9432220F9039
:1044A000039401FC9058E9EDF0E00C94612357FD72
:1044B0009058440F551F59F05F3F71F04795880F92
:1044C00097FB991F61F09F3F79F087950895121629
:1044D00013061406551FF2CF4695F1DF08C01616D5
:1044E00017061806991FF1CF869571056105089486
:1044F0000895E894BB2766277727CB0197F908959D
:104500000E94A52108F48FEF08959B01AC0160E0A3
:1045100070E080E89FE30C94C0200E94A0220C94DD
:1045200032220E94F92138F00E94002220F09523C7
:1045300011F00C94C9210C94CF2111240C947A22EF
:104540000E94572270F3959FC1F3950F50E0551FBD
:10455000629FF001729FBB27F00DB11D639FAA27D8
:10456000F00DB11DAA1F649F6627B00DA11D661F27
:10457000829F2227B00DA11D621F739FB00DA11D48
:10458000621F839FA00D611D221F749F3327A00D02
:10459000611D231F849F600D211D822F762F6A2F9E
:1045A00011249F5750409AF0F1F088234AF0EE0F03
:1045B000FF1FBB1F661F771F881F91505040A9F730
:1045C0009E3F510580F00C94C9210C947A225F3FE4
:1045D000E4F3983ED4F3869577956795B795F7956C
:1045E000E7959F5FC1F7FE2B880F911D96958795E4
:1045F00097F908959F930E9409220F9007FCEE5FA0
:104600000C94432219F416F40C94CF210C944C23EF
:104610000E945F22B8F39923C9F3B6F39F57550B55
:1046200087FF0E945A230024A0E640EA90018058A8
:104630005695979528F4805C660F771F881F20F0A9
:1046400026173707480730F4621B730B840B2029A9
:1046500031294A2BA69517940794202531254A27FE
:1046600058F7660F771F881F20F02617370748076F
:1046700030F4620B730B840B200D311D411DA0958E
:1046800081F7B901842F9158880F969587950895E1
:104690009B01AC010C948D229F3F31F0915020F48E
:1046A000879577956795B795880F911D969587950E
:1046B00097F9089591505040660F771F881FD2F7E1
:1046C00008959F938F937F936F93FF93EF939B0135
:1046D000AC010E948D22EF91FF910E94D2212F9177
:1046E0003F914F915F910C948D22AA1BBB1B51E10E
:1046F00007C0AA1FBB1FA617B70710F0A61BB70B52
:10470000881F991F5A95A9F780959095BC01CD01F6
:10471000089597FB072E16F4009407D077FD09D073
:104720000E94752307FC05D03EF4909581959F4F1C
:104730000895709561957F4F08950E94C81F332397
:1047400012F48A1B9B0B0C94A7230E94C81FB7FF6F
:104750000895821B930B0895EE0FFF1F0590F491AF
:08476000E02D0994F894FFCF4D
:1047680010C3F5C8BF010000C8420000C8420000DD
:1047780080430000804364000300D0074000FFFF2F
:10478800FFFF00E10000000000000100000000C180
:1047980080810000000000000048056F0669055E82
:1047A80005AF056D058B05000000009F090A07523B
:0447B8000B510B0096
:00000001FF
